:10000000A0019D2990002408840022081021841357
:100010000005181C2206031920281008031D1828A3
:100020001608FF3E031C21280A3025211608212826
:10003000100AFF3003192028100B20281708212848
:100040009909990C9829A016A01EA01220192D28F4
:10005000FE39A100201503109829201A3528920096
:1000600020164C2003183A281208532003183A2867
:10007000A01E982945206A2020112012A0112408D2
:1000800084002208841780044B2824088400220955
:1000900080058417800508003F206A2045206620DF
:1000A0002108A01901388E0008308F008E0D03182A
:1000B0003F20031C45206A2066208F0B56283F20D6
:1000C0006A202408840022080005FF3E25088400D9
:1000D000230948282508840023088004841723095D
:1000E00080054B2891019000A11727308F00103018
:1000F000852003308F00E83085208F016430852013
:100100008F010A308520100890288E0011088D007C
:1001100010088C0061210C08031DA113A11B08000D
:10012000303E9328040893008611861086108316AB
:100130008611861086100F30860583121308A018CA
:10014000BF283A308D009830332133309200D320CD
:1001500013308D0088303321D32064303221D320F6
:100160006430322122309200D3202830BE200C305F
:10017000BE200630BE20A0141308BF282014920011
:10018000201CCD288610033C031CD228D220073027
:100190008D00D0303321031408002014FE3C0319D5
:1001A00098298614201C201086150F308605120809
:1001B000F03986048611920E2018D328323032216D
:1001C00003140800A11315080319A11705309400A2
:1001D00027308F001030F82003308F00E830F820EF
:1001E0008F016430F8208F010A30F8201008FF28B2
:1001F0008E0011088D0010088C0061210C088C0005
:1002000094030319A11315080319092914020318EB
:1002100008000C08031DA113A11B0800303E932900
:10022000841780049829890083160814831208080B
:10023000982988008316081555308900AA3089004E
:10024000881488182129081198298F018E00FF3001
:100250008E07031C8F07031C982903308D00DF30A5
:10026000332127298D01E83E8C008D09FC30031CC9
:100270003C298C07031839298C0764008D0F392914
:100280000C1842298C1C46290000462908008E00C3
:10029000023051298E00063051298F018E00043022
:1002A000512994000F080D02031D58290E080C0255
:1002B000043003180130031902301405031DFF3008
:1002C000982991019001103092000D0D900D910D23
:1002D0000E0890020F08031C0F0F910203187729D4
:1002E0000E0890070F0803180F0F910703108C0DCD
:1002F0008D0D920B65290C089829103094008D0102
:100300008C01930C920C031C8B290E088C070F0890
:1003100003180F0F8D078D0C8C0C910C900C940B07
:1003200081291008982984001D088A001C08820071
:1003300083130313831264000800831605148514C5
:100340000515051685158312C230B4008030AE0045
:100350003E30AF000130BB0064302521061183160A
:100360000611FE30831293200130932054309320E5
:1003700058309320203093204130932054309320E4
:10038000563093202030932032309320FE3093203B
:10039000C03093202E309320333093204730932069
:1003A000483093207A309320203093207630932069
:1003B00031309320BC014130B200B30103308F00D3
:1003C000E83026213C081321B00001303C079E0094
:1003D0009F019F0D1E081321B1002E083007AC00AD
:1003E0002F080318013E3107AD000630A40001308C
:1003F000A2000630A5000230A300340825202D08F5
:1004000025202C0825208E302320C722F2220130FF
:100410008F00F43026210530A4000830A200980196
:10042000FF30960097010130990039080220B90089
:1004300003186B2A0530A4000830A2000130980090
:10044000FF3096009701013099003A080220BA0067
:100450000318702A0530A4000130A20098010A3068
:100460009600023097000130990035080220B5004F
:100470000318762A0530A4000230A20098010A3041
:100480009600023097000130990036080220B6002D
:100490000318872A0530A4000430A2009801FF3019
:1004A000960097010130990038080220B80003181F
:1004B000502B0530A4001030A2009801FF309600A8
:1004C00097010130990037080220B7000318A52AC8
:1004D000643025210B2ABC014130B200B301E2296E
:1004E0000230BC004230B200B301E2293B08B00741
:1004F0000318B10A30088C0031088D0014308F00C9
:1005000050304A21031D862AB001B101ED2930087F
:100510008C0031088D003B084D21031DA22A3008B4
:100520008C0031088D008F0100304721031D9D2A6A
:100530003B08B002031CB103ED295030B000143069
:10054000B100ED29B001B101ED2964003B08503C38
:100550000319BB2A64003B08083C0319C12A3B0865
:100560009200930102308E008F017D21BB001F237A
:10057000C722F2220B2A0130BB001F23C722F2221E
:100580000B2A5030BB001F23C722F2220B2A8030D7
:100590002C02A6003E30031C013E2D02A7002608B7
:1005A0008C0027088D0008308E008F016121A80083
:1005B0000D08A90026088C0027088D0008308E0041
:1005C0008F01612110089E0011089F007D3092006C
:1005D00093011E088E001F088F007D21AA001108BC
:1005E000AB000800FE3093200130932002307220CF
:1005F00003309500280890002908910092309C0053
:100600009D01E2202E309320033095002A089000AF
:100610002B08910092309C009D01E220FE30932037
:10062000C0309320203093204D30932048309320C9
:100630007A30932020309320320893200800FE3037
:1006400093200130932050309320613093207330F9
:100650009320203093206430932065309320203005
:100660009320FE309320C03093207D309200930180
:100670003B088E008F017D219E0011089F001F08FE
:1006800091001E087320203093206B309320483057
:1006900093207A30932005308F00DC30262108002B
:1006A0003C0889003008192101303C079E009F0159
:1006B0009F0D1E08890031081921FE30932001305A
:1006C00093204D309320453093204D3093204F3070
:1006D000932052309320493093205330932045305B
:1006E0009320FE309320C03093202030932073302D
:1006F000932075309320723093202030932032085D
:10070000932005308F00DC302621C722F2220B2AED
:02400E00F53F7C
:08420000A000090000000A0003
:00000001FF
